:1000000010C02AC029C028C027C026C025C024C0CF
:1000100023C022C021C020C01FC01EC01DC01CC0E4
:100020001BC011241FBECFE5D1E0DEBFCDBF10E065
:10003000A0E6B0E0E0EBF0E002C005900D92A23641
:10004000B107D9F720E0A2E6B0E001C01D92A436C6
:10005000B207E1F70ED02AC0D3CF369A3699FECF39
:1000600084B195B1089582E087B993E896B981B9D2
:100070000895D39AD49AD698F6DFCE9B02C0DB9827
:1000800001C0DB9AEADF90936300809362002091C5
:10009000620030916300809160009091610082174E
:1000A000930710F4DC98E9CFDC9AE7CFF894FFCF00
:0200B00000024C
:00000001FF
